:020000000528D1
:06000A008316FF308600A2
:10001000FE308500D830810020308B008312003004
:100020009000910092009300940095009600970034
:10003000980099009A009B009C009C009E009F00E5
:10004000A000A100A200A200A300A400A500A60099
:10005000A700A800A900AA00AB00AC00AD00AE004C
:10006000AF00B000B100B200B300B400B500B600FC
:10007000B700B800B900BA00BB00BC00BC00BE00AD
:10008000BF00C000C100C200C300C400C500C6005C
:10009000C700C800C900CA00CB00CC00CD00CE000C
:1000A000CF00851C63281030840003118519851D3D
:1000B000572806088000840A0408503A0319632868
:1000C000851960285628051400000000000005145A
:1000D000000000000000051000000000000000000B
:1000E0000000000000000000000000000000000010
:1000F0000000000000000000000000000000000000
:1001000000000000000000000000000000000000EF
:1001100000000000000000000000000000000000DF
:1001200000000000000000000000000000000000CF
:1001300000000000000000000000000000000000BF
:1001400000000000000000000000000000000000AF
:10015000000000000000000000000000000000009F
:10016000000000000000000000000000000000008F
:10017000000000000000000000000000000000007F
:10018000000000000000000000000000000000006F
:10019000000000000000000000000000000000005F
:1001A000000005140000000000000514000000001D
:1001B000000005100000000000000000000000002A
:1001C000000000000000000000000000000000002F
:1001D000000000000000000000000000000000001F
:1001E000000000000000000000000000000000000F
:1001F00000000000000000000000051400000000E6
:1002000000000514000000000000051400000000BC
:1002100000001030840000080510000000000000FD
:100220008500800C000800008500800C000800009C
:100230008500800C000800008500800C000800008C
:100240008500800C000800008500800C000800007C
:100250008500800C000800008500800C0008800CE0
:10026000051400000000000005140000000000005C
:100270000514000000000000031100000000000051
:0E0280006400840A0408503A031D0B2951281B
:02400E00F13F80
:00000001FF
